:0200000480007A
:100000009710000093800000171100001301810178
:1000100083A1000013021000B70200809382F2FF58
:100020001303F0FF930300003704008033B2410054
:10003000B3B2510033B36100B3B3710033B4810084
:100040002320310023224100232451002326610074
:1000500023287100232A8100971000009380C0FAA2
:1000600017110000130181FD03A400009304100088
:10007000370500801305F5FF9305F0FF1306000018
:10008000B7060080B33494003335A400B335B40010
:100090003336C400B336D4002320810023229100DC
:1000A0002324A1002326B1002328C100232AD10044
:1000B00097100000938080F517110000130181F95B
:1000C00083A6000013071000B70700809387F7FF8F
:1000D0001308F0FF930800003709008033B7E600EB
:1000E000B3B7F60033B80601B3B8160133B9260129
:1000F0002320D1002322E1002324F1002326010143
:1001000023281101232A210197100000938040F039
:1001100017110000130181F503A9000093091000D5
:10012000370A0080130AFAFF930AF0FF130B00004E
:10013000B70B0080B3393901333A4901B33A590159
:10014000333B6901B33B7901232021012322310193
:10015000232441012326510123286101232A71010F
:1001600097100000938000EB17110000130181F13C
:1001700083AB0000130C1000B70C0080938CFCFFC5
:10018000130DF0FF930D0000370E008033BC8B0180
:10019000B3BC9B0133BDAB01B3BDBB0133BECB01CF
:1001A0002320710123228101232491012326A1010F
:1001B0002328B101232AC101171D0000130DCDE52D
:1001C000971D0000938D8DED83200D001301F0FF2E
:1001D00033B0200023A00D0023A21D0023A42D0076
:1001E000971F0000938F4FEC930010001301F07FD6
:1001F0009301F0FF130200009302008033331000DC
:10020000B333200033343000B33440003335500072
:10021000B3B5000033360100B3B601003337020036
:10022000B3B7020023A06F0023A27F0023A48F0096
:1002300023A69F0023A8AF0023AABF0023ACCF00B2
:1002400023AEDF0023A0EF0223A2FF02971F0000CE
:10025000938F0FE893011000B330300033B13000BA
:10026000333E3100B33E3E0033BF3E0023A01F00AB
:1002700023A22F0023A4CF0123A6DF0123A8EF018F
:1002800017150000130505DA97150000938585E51D
:10029000370610F01306C6F26306B5028326C500C2
:1002A0002320D600832685002320D6008326450000
:1002B0002320D600832605002320D6001305050140
:1002C0006FF09FFD370510F0130505F223200500A0
:0402D000000000002A
:101000000000000001000000FFFFFFFFFFFFFF7F67
:10101000000000800100000000000000000000004F
:10102000FFFFFFFFFFFFFFFFFFFFFFFFFFFFFFFFD0
:10103000FFFFFFFFFFFFFFFFFFFFFFFFFFFFFFFFC0
:10104000FFFFFFFFFFFFFFFFFFFFFFFFFFFFFFFFB0
:10105000FFFFFFFFFFFFFFFFFFFFFFFFFFFFFFFFA0
:10106000FFFFFFFFFFFFFFFFFFFFFFFFFFFFFFFF90
:10107000FFFFFFFFFFFFFFFFFFFFFFFFFFFFFFFF80
:10108000FFFFFFFFFFFFFFFFFFFFFFFFFFFFFFFF70
:10109000FFFFFFFFFFFFFFFFFFFFFFFFFFFFFFFF60
:1010A000FFFFFFFFFFFFFFFFFFFFFFFFFFFFFFFF50
:1010B000FFFFFFFFFFFFFFFFFFFFFFFFFFFFFFFF40
:1010C000FFFFFFFFFFFFFFFFFFFFFFFFFFFFFFFF30
:1010D000FFFFFFFFFFFFFFFFFFFFFFFFFFFFFFFF20
:040000058000000077
:00000001FF
